:020000001C28BA
:1000080005288D00030E83018C0004088E008401EE
:100018000A088F008A010B1851288B1844280F08EA
:100028008A000E0884000C0E83008D0E0D0E090048
:1000380040306200003086008501113066000030D3
:100048006500033056209501060898308B00951CF2
:100058002B2882300102031C2D28951086102B288E
:100068000139031D8514382839288510523090002D
:10007800900B3C28080029309000900B412808007C
:100088003F20061C4F280130342008309400060811
:100098003420940B4B288B10132886148101951457
:1000A8000B10132890005B20900B57280800643031
:1000B80091006120910B5D280800FA3092006428B5
:0C00C800652866280000920B63280800E1
:02400E00F23F7F
:00000001FF
